S01D000062696E2F6F70656E626C745F73746D3332683734332E737265638D
S3150800000000000220050400085504000855040008ED
S3150800001055040008550400085504000800000000AF
S315080000200000000000000000000000005504000861
S31508000030550400080000000055040008550400088F
S31508000040550400085504000855040008550400081E
S31508000050550400085504000855040008550400080E
S3150800006055040008550400085504000855040008FE
S3150800007055040008550400085504000855040008EE
S3150800008055040008550400085504000855040008DE
S3150800009055040008550400085504000855040008CE
S315080000A055040008550400085504000855040008BE
S315080000B055040008550400085504000855040008AE
S315080000C0550400085504000855040008550400089E
S315080000D0550400085504000855040008550400088E
S315080000E055040008550400080000000055040008DF
S315080000F0550400085504000855040008550400086E
S31508000100550400085504000855040008550400085D
S31508000110550400085504000855040008550400084D
S31508000120550400085504000855040008550400083D
S31508000130550400085504000855040008550400082D
S3150800014000000000000000000000000000000000A1
S31508000150550400085504000855040008550400080D
S3150800016055040008550400085504000855040008FD
S31508000170550400085504000855040008000000004E
S3150800018055040008550400085504000855040008DD
S3150800019055040008550400085504000855040008CD
S315080001A055040008550400085504000855040008BD
S315080001B055040008550400085504000855040008AD
S315080001C0550400085504000855040008550400089D
S315080001D0550400085504000855040008550400088D
S315080001E0550400085504000855040008550400087D
S315080001F0550400085504000855040008550400086D
S31508000200550400085504000855040008550400085C
S31508000210550400085504000855040008550400084C
S31508000220550400085504000855040008000000009D
S31508000230550400085504000800000000550400088D
S31508000240550400085504000855040008550400081C
S31508000250550400085504000855040008550400080C
S3150800026055040008550400085504000855040008FC
S31508000270550400085504000855040008000000004D
S31508000280550400085504000855040008000000003D
S30D080002900000000055040008F7
S3150800029810B5054C237833B9044B13B10448AFF3AA
S315080002A800800123237010BDF00400200000000020
S315080002B8B05C000808B5034B1BB103490348AFF304
S315080002C8008008BD00000000F4040020B05C0008A7
S315080002D870B50D4E0D4D761BB61006D000240134A8
S315080002E855F8043B9847A642F9D1094E094D761B9D
S315080002F805F0DAFCB61006D00024013455F8043B9C
S315080003089847A642F9D170BD285F0008285F0008FB
S31508000318305F0008285F0008024B13B1024800F056
S3150800032805B870470000000041030008002301468D
S315080003381A46184600F01EB838B50A4C0A4D641B0A
S31508000348A4100AD004F18043013B05EB8305013C60
S3150800035855F804399847002CF9D1BDE8384005F016
S31508000368A9BC00BF345F0008305F0008704700BFAB
S31508000378704700BF2DE9F0411E4C05462068904697
S315080003881F460E46FFF7F2FF1B4B1A68D2F848318C
S3150800039833B35A6820681F2A27DC4DB9911C0132E5
S315080003A85A6043F82160FFF7E3FF0020BDE8F081B3
S315080003B803EB82010124C1F8888004FA02FED3F807
S315080003C88841022D44EA0E0CC3F888C1C1F80871A1
S315080003D8E4D1D3F88C114EEA0104C3F88C41DDE761
S315080003E802F5A673C2F84831D3E7FFF7C1FF4FF005
S315080003F8FF30DBE728040020145D0008DFF834D056
S31508000408002103E00C4B5B58435004310B480C4B56
S3150800041842189A42F6D30B4A02E0002342F8043BF4
S31508000428094B9A42F9D300F033FDFFF751FF04F060
S315080004383FF8704700000220345F000800000020DB
S31508000448F0040020F004002034190020FEE710B557
S3150800045813460222C0F89422C36103620A460021A1
S3150800046804F0D4FA002010BD08B513460A46002140
S3150800047804F0CCFA002008BD08B513460A46002140
S3150800048804F0CCFA002008BD08B50423C0F8943255
S3150800049800231A46194604F0B9FA002008BD08B51B
S315080004A80523C0F8943200231A46194604F0B6FA0A
S315080004B8002008BD002302781AB10133DBB20130E7
S315080004C8F9E71846704708B54B88012B00D008BDD0
S315080004D8C0F8A432FFF7D8FFF9E70B7803704B7812
S315080004E843708B78CA7803EB022343800B794A79E1
S315080004F803EB022383808B79CA7903EB0223C38033
S31508000508704710B50446802104F068FA0021204691
S3150800051804F064FA10BD30B583B005460C460023CE
S31508000528ADF806304A88130A013B062B00F2A48068
S31508000538DFE803F004182CA2A2869300D0F8B0329C
S315080005481B680DF10601007C9847BDF806201AB10C
S31508000558E388002B40F09480E388002B00F09A800B
S3150800056803B030BD037C43B9D0F8B4329B6A0DF1A9
S315080005780600984702234370E7E7D0F8B432DB6AE7
S315080005880DF10600984702234370DEE7D2B2052A22
S3150800059852D8DFE802F003101D2A3744D0F8B032E3
S315080005A85B6823B10DF10601007C9847CDE7214623
S315080005B8FFF7A7FFD4E7D0F8B0329B6823B10DF14F
S315080005C80601007C9847C0E72146FFF79AFFC7E768
S315080005D8D0F8B032DB6823B10DF10601007C9847E4
S315080005E8B3E72146FFF78DFFBAE7D0F8B0321B69A3
S315080005F823B10DF10601007C9847A6E72146FFF7C7
S3150800060880FFADE7D0F8B0325B6923B10DF106017A
S31508000618007C984799E72146FFF773FFA0E7D0F8CB
S31508000628B0329B6923B10DF10601007C98478CE727
S315080006382146FFF766FF93E72146FFF762FF8FE734
S31508000648037C33B9D0F8B4325B6B0DF106009847D2
S315080006587BE72146FFF755FF82E7037C43B9D0F8C5
S31508000668B4321B6B0DF106009847072343706CE7F5
S315080006782146FFF746FF73E72146FFF742FF6FE774
S315080006889A4228BF1A46ADF8062001462846FFF7BB
S31508000698DEFE61E72846FFF7F7FE61E738B5044648
S315080006A88B88F3B9CB88E3B94B887F2B19D803F025
S315080006B87F0590F89C32032B0CD080F89E52294669
S315080006C804F09CF92046FFF7DFFE35B1022384F8CB
S315080006D89C3209E0FFF715FF06E0012384F89C32EF
S315080006E802E02046FFF70DFF38BD000038B504467E
S315080006F80D468978284B197001290ED890F89C322E
S31508000708022B0ED0032B21D02946FFF7FAFE224BDF
S315080007181978204600F072FA02E02946FFF7F1FE3A
S3150800072838BD81B14160032380F89C3200F059FA3C
S31508000738022803D02046FFF7A7FEF1E729462046F8
S31508000748FFF7DFFEECE7FFF79FFEE9E789B14368A5
S3150800075899421DD0D9B200F051FA0F4B1978616049
S31508000768204600F03EFA02280DD02046FFF78CFEF8
S31508000778D6E7022380F89C32416000F03FFA20460B
S31508000788FFF782FECCE729462046FFF7BAFEC7E7F9
S31508000798FFF77AFEC4E700BF0C05002008B5CB882A
S315080007A8012B0CD190F89C325AB29AB1022B09D96E
S315080007B8032B0FD10122011DFFF749FE01E0FFF7C0
S315080007C8A0FE08BD0146002341F8083F0122FFF7AD
S315080007D83EFEF6E7FFF795FEF3E708B590F89C3274
S315080007E8013B022B12D8CB88022B0CD10123C360FC
S315080007F8D0F8A4320BB10323C360022200F10C011E
S31508000808FFF725FE08BDFFF77CFEFBE7FFF779FE35
S31508000818F8E708B590F89C32013B022B09D84B88B3
S31508000828012B00D008BD0023C0F8A432FFF72CFE20
S31508000838F8E7FFF766FEF5E708B50B7803F06003F7
S31508000848202B05D0402B03D043B1FFF75AFE03E00F
S31508000858D0F8B4329B689847002008BD4B78092B16
S315080008681BD8DFE803F011171A141A08051A0E0B15
S31508000878FFF751FEF0E7FFF711FFEDE7FFF736FF41
S31508000888EAE7FFF78BFFE7E7FFF7A7FFE4E7FFF7D6
S315080008981AFEE1E7FFF7BDFFDEE7FFF732FEDBE703
S315080008A838B505460C460B7803F06003202B06D0AE
S315080008B8402B04D01BB1FFF724FE002038BD95F85D
S315080008C89C32013B022B16D82379012B0ED8D5F872
S315080008D8B4329B68214628469847E388002BECD112
S315080008E80028EAD12846FFF7CFFDE6E7214628463D
S315080008F8FFF707FEE1E721462846FFF702FEDCE791
S3150800090838B504468A880B7803F06003202B08D08C
S31508000918D0B2402B05D05BB12046FFF7F2FD002088
S3150800092805E0D4F8B4329B6820469847002038BDBD
S31508000938202B13D04B78012B43D05DB2002D73D0F2
S31508000948032B40F0F78094F89C32022B0CD0032B2B
S3150800095821D02046FFF7D5FD0020E8E7D4F8B432C1
S315080009689B6820469847E2E7B0F1800318BF012341
S31508000978002808BF00234BB10146204604F02EF88C
S315080009888021204604F02AF80020D0E72046FFF701
S31508000998B8FD0020CBE74B884BB9B0F1800318BFE8
S315080009A80123002808BF00230BB1CB8823B12046B2
S315080009B8FFF76AFD0020BAE70146204604F00EF85C
S315080009C8F5E794F89C32022B06D0032B1BD0204659
S315080009D8FFF797FD0020AAE7B0F1800318BF0123A7
S315080009E8002808BF00234BB10146204603F0F6FF4E
S315080009F88021204603F0F2FF002098E72046FFF7FB
S31508000A0880FD002093E74B88002B40F0988010F073
S31508000A187F0F04D12046FFF737FD002087E70146F8
S31508000A28204603F0E3FFF5E794F89C32022B06D03C
S31508000A38032B2FD02046FFF764FD002077E7B0F197
S31508000A48800318BF0123002808BF00239BB912F0AA
S31508000A58800F15D100F07F0000EB8000830003F5B6
S31508000A68A8712144043100250D6002222046FFF7AB
S31508000A78EEFC28465BE72046FFF743FD002056E7CD
S31508000A8800F07F0000EB8000830003F11001214489
S31508000A980431E8E752B2002A24DB00F00F0303EB1F
S31508000AA883039D002544D5F858314BB3002A2CDB1F
S31508000AB800F07F0202EB8202930003F5A87525442D
S31508000AC80435802814BF00230123002808BF012302
S31508000AD82BB300232B60022229462046FFF7B7FCD2
S31508000AE8002024E700F00F0303EB83039D00254449
S31508000AF8AB69002BDAD12046FFF703FD002016E77D
S31508000B082046FFF7FEFC002011E700F07F0202EB03
S31508000B188202930003F1100525440435D1E70146FE
S31508000B28204603F007FF10B101232B60D3E7002303
S31508000B382B60D0E72046FFF7E4FC0020F7E6002004
S31508000B48F5E6C0B170B50D4616460446FFF7B2FC81
S31508000B58013040003080287003236B700223217807
S31508000B6841B101345A1CD2B2E9540233DBB200212E
S31508000B78A954F4E770BD704798B108B50346D0F88C
S31508000B88B40210B10020C3F8B40209B1C3F8B01210
S31508000B981846012380F89C32027003F08FFE002065
S31508000BA808BD0220704710B50446012380F89C3218
S31508000BB8D0F8B4325B6801799847204603F0F3FE0B
S31508000BC8204603F0E0FE002010BD19B1C0F8B412A3
S31508000BD8002070470220704708B503F0DCFE0020A5
S31508000BE808BD08B5D0F8B43233B11B68984708B9B8
S31508000BF8002008BD0220FCE70220FAE708B5D0F86D
S31508000C08B4325B689847002008BD38B5044600F535
S31508000C182A752846FFF761FC0123C4F89432B4F80C
S31508000C28AE32C4F8983294F8A81201F01F03012BC3
S31508000C380FD05AB23AB1022B10D001F080012046E3
S31508000C4803F0CCFE03E029462046FFF7F5FD002011
S31508000C5838BD29462046FFF723FEF8E729462046E9
S31508000C68FFF74EFEF3E738B50446A9BB1046D4F895
S31508000C789432032B03D0052B25D0002038E0D4F86E
S31508000C886031D4F8642193420DD99B1AC4F86031AF
S31508000C989A4206D99AB201462046FFF7EDFB00208C
S31508000CA826E092B2F7E7D4F8B4321B691BB194F878
S31508000CB89C22032A04D02046FFF7E6FB002017E00B
S31508000CC820469847F7E70025C4F89452294620464F
S31508000CD803F084FE28460BE00A46D0F8B4329B692E
S31508000CE83BB190F89C12032905D111469847002074
S31508000CF838BD0220FCE70220FAE710B504460029A9
S31508000D0856D11046D4F89432022B09D0002B18BFB6
S31508000D18042B44D094F8A032012B45D0002010BDEE
S31508000D28236A626A93421BD8E169B1FBF2F302FBB4
S31508000D3813132BB98A4203D8D4F8983299421DD38B
S31508000D48D4F8B432DB681BB194F89C22032A23D062
S31508000D588021204603F042FE2046FFF7A0FBD9E78C
S31508000D689A1A226292B201462046FFF77DFB0023B3
S31508000D781A461946204603F051FECBE700221146CB
S31508000D882046FFF771FB0021C4F898120B460A465D
S31508000D98204603F043FEBDE720469847D8E780215A
S31508000DA8204603F01BFEB5E7002084F8A002B6E744
S31508000DB80A46D0F8B4325B693BB190F89C1203290D
S31508000DC805D1114698470020A9E70220A7E702207F
S31508000DD8A5E770B5044640230022114603F0EBFD4B
S31508000DE80125C4F858514026C4F8646133460022E0
S31508000DF88021204603F0DFFDA561666284F89C52CF
S31508000E080023C4F894326360C4F8A432D4F8B8321C
S31508000E182BB1D4F8B4325B680021204698470020E5
S31508000E2870BD01740020704790F89C3280F89D3296
S31508000E38042380F89C320020704790F89C32042BD3
S31508000E4801D00020704790F89D3280F89C32F8E768
S31508000E5808B590F89C32032B01D0002008BDD0F8BD
S31508000E68B432DB69002BF8D09847F6E700207047BC
S31508000E78002070470020704708B5012280F89C2298
S31508000E88D0F8B422526801799047002008BD0000BE
S31508000E98184AD2F8883043F47003C2F88830164BDB
S31508000EA81A6842F001021A6000221A611868134982
S31508000EB8014019609A61DA611A629A62DA621A63FB
S31508000EC85A639A63DA631A645A64196821F48021A2
S31508000ED819601A660A4B1A680A4B1340B3F1005F81
S31508000EE802D2094B01221A60024B4FF000629A603F
S31508000EF8704700BF00ED00E0004402587FEDF6EAAF
S31508000F080010005C0000FFFF0881005110B5164B61
S31508000F186FF00042DA670024DC674FF0FF32C3F847
S31508000F288020C3F88040C3F88420C3F88440C3F8F7
S31508000F388820C3F88840C3F88C20C3F88C40C3F8C7
S31508000F489020C3F89040C3F89420C3F89440C3F897
S31508000F589820C3F89840C3F89C20C3F89C4003F02F
S31508000F685FFB204610BD00BF00440258104B1B7893
S31508000F780BB90120704710B504464FF47A70B0FBD8
S31508000F88F3F30C4A1068B0FBF3F002F095FA68B967
S31508000F980F2C01D901200AE0002221464FF0FF3024
S31508000FA802F058FA044B1C60002000E0012010BD2E
S31508000FB8340400202C0400203804002010B503202F
S31508000FC802F036FA02F06AF80F498B69C3F303236D
S31508000FD80E4AD35C03F01F03D8408B6903F00F034E
S31508000FE8D35C03F01F0320FA03F3094A1360094B7D
S31508000FF818600020FFF7BAFF10B10124204610BD7B
S31508001008044603F05DFAF9E700440258185D00083B
S31508001018300400202C04002038B5044604F040F8B3
S315080010280546B4F1FF3F02D0044B1B781C4404F074
S3150800103837F8401BA042FAD338BD00BF3404002055
S31508001048204A136843F0010313601E4B1B6813F00C
S31508001058040FFAD01B4B00221A6119681A4A0A406B
S315080010681A60184B1B6813F0007FFAD1154B1B68DA
S3150800107813F0006FFAD1134B1B6813F0005FFAD10F
S31508001088104B00229A61DA611A621049996210496E
S31508001098D962104919635A639963DA6319645A64F9
S315080010A8196821F4802119601A66996E40F2FF7250
S315080010B80A439A66D3F8D02042F48032C3F8D0207F
S315080010C8704700BF0044025845EDF6EA00020202DE
S315080010D80000FF018002010107EE900AF8EE676A30
S315080010E807EE901AF8EE677A86EEA77A07EE902A40
S315080010F8F8EE677A06EE903AF8EE666A9FED096AA0
S3150800110866EE866A77EEA67A27EE277ADDED007A06
S31508001118F8EE677AC7EE276AFCEEE67A17EE900AC3
S31508001128704700BF000000392DE9F04182B03E4BF8
S315080011389B6A03F00303012B24D0BBB1022B28D0EA
S3150800114800270023036043608360374B9E6AC6F313
S3150800115805161A6BC2F30802551CDB6A13F0010F51
S3150800116824D0314B5B6BC3F3CC0821E02E4B1B68AC
S3150800117813F0040F14D02C4B1B68C3F3C1032B4F71
S31508001188DF40DEE7284B1B6813F4807F0AD1002767
S31508001198D7E7254B1B6813F4003F05D10027D0E78E
S315080011A80027CEE7224FCCE7224FCAE74FF00008C0
S315080011B8002E36D004461C4BDB6A13F4803F0CD04D
S315080011C8194B1B6BC3F346230133009343462A4640
S315080011D831463846FFF780FF2060134BDB6A13F465
S315080011E8003F0CD0104B1B6BC3F306430133009327
S315080011F843462A4631463846FFF76EFF60600A4B73
S31508001208DB6A13F4802F0CD0074B1B6BC3F30663FA
S315080012180133009343462A4631463846FFF75CFFB2
S31508001228A06002B0BDE8F081004402580090D003DF
S3150800123800093D0000127A002DE9F04182B03E4BC4
S315080012489B6A03F00303012B24D0BBB1022B28D0D9
S3150800125800270023036043608360374B9E6AC6F302
S3150800126805369A6BC2F30802551CDB6A13F0100F91
S3150800127824D0314BDB6BC3F3CC0821E02E4B1B681B
S3150800128813F0040F14D02C4B1B68C3F3C1032B4F60
S31508001298DF40DEE7284B1B6813F4807F0AD1002756
S315080012A8D7E7254B1B6813F4003F05D10027D0E77D
S315080012B80027CEE7224FCCE7224FCAE74FF00008AF
S315080012C8002E36D004461C4BDB6A13F4002F0CD0CC
S315080012D8194B9B6BC3F346230133009343462A46AF
S315080012E831463846FFF7F8FE2060134BDB6A13F4DD
S315080012F8801F0CD0104B9B6BC3F306430133009336
S3150800130843462A4631463846FFF7E6FE60600A4BEA
S31508001318DB6A13F4001F0CD0074B9B6BC3F30663F9
S315080013280133009343462A4631463846FFF7D4FE2A
S31508001338A06002B0BDE8F081004402580090D003CE
S3150800134800093D0000127A002DE9F04182B0424BAF
S315080013589B6A03F00303012B24D0BBB1022B28D0C8
S31508001368002500230360436083603B4B9C6AC4F3F3
S3150800137805541A6CC2F30802561CDB6A13F4807FFC
S3150800138824D0354B5F6CC7F3CC0720E0324B1B687B
S3150800139813F0040F14D0304B1B68C3F3C1032F4D49
S315080013A8DD40DEE72C4B1B6813F4807F0AD1002545
S315080013B8D7E7294B1B6813F4003F05D10025D0E76A
S315080013C80025CEE7264DCCE7264DCAE700272B1C75
S315080013D818BF0123002C08BF0023002B39D08046EC
S315080013E81D4BDB6A13F4800F0DD01B4B1B6CC3F324
S315080013F84623013300933B46324621462846FFF7E3
S315080014086BFEC8F80000144BDB6A13F4000F0DD006
S31508001418114B1B6CC3F30643013300933B46324614
S3150800142821462846FFF758FEC8F804000A4BDB6A27
S3150800143813F0807F0DD0084B1B6CC3F3066301338A
S3150800144800933B46324621462846FFF745FEC8F82C
S31508001458080002B0BDE8F081004402580090D003A5
S3150800146800093D0000127A00154B1B6903F0380382
S31508001478182B0ED8DFE803F00F0D0D0D0D0D0D0D09
S31508001488210D0D0D0D0D0D0D160D0D0D0D0D0D0D59
S315080014981800002070470A4B1B68C3F3C1030948A4
S315080014A8D84070470848704700B585B001A8FFF7C7
S315080014B83BFE019805B05DF804FB0448704700BF79
S315080014C8004402580090D00300127A0000093D0033
S315080014D8044B9B6903F00F03034AD35C03F01F030D
S315080014E8D840704700440258285D0008044BDB6959
S315080014F8C3F30213034AD35C03F01F03D8407047AB
S3150800150800440258285D0008044BDB69C3F302232C
S31508001518034AD35C03F01F03D840704700440258B7
S31508001528285D000800B585B0C2B24F4BD358020EE5
S31508001538C0F304218A401340CB4040EA03404B4B92
S31508001548984228D033D8A3F58133A3F580739842F7
S3150800155866D019D8A3F58033984251D003F540735D
S3150800156898420FD1FFF780FF414B9B69C3F30323CA
S31508001578404AD35C03F01F03D840FFF7A9FFFFF7DB
S31508001588C3FF24E0002022E03B4B984248D003F5ED
S315080015987D43984209D1364B1B6813F0005F59D032
S315080015A801A8FFF7D1FE029811E000200FE0334B9F
S315080015B898423FD00ED9324B984242D003F5407331
S315080015C898423ED0A3F58033984233D0002005B020
S315080015D85DF804FBA3F58033984203D003F54073FE
S315080015E898420BD1224B1B6813F0040F34D0204BBA
S315080015F81B68C3F3C1032348D840E8E70020E6E799
S31508001608FFF732FF1A4B9B69C3F30323194AD35CC6
S3150800161803F01F03D840FFF75BFFFFF767FFD6E71E
S31508001628134B1B6813F0006F12D001A8FFF704FECE
S315080016380298CCE70E4B1B6813F4807F0ED1002066
S31508001648C5E70B4B1B6F13F0020F09D10020BEE745
S315080016580020BCE70020BAE70020B8E70A48B6E742
S315080016684FF40040B3E700BF4C440258080302078A
S3150800167800440258285D0008080301070800040703
S31508001688080005070090D00300093D0030B4446BF4
S315080016980268D2F88410704B194041EA8401C2F8EE
S315080016A884100268D2F8841021F47F01856B41EA18
S315080016B80541C2F88410826B22440468D4F888105D
S315080016C8194041EA8201C4F888100468D4F88810D9
S315080016D821F4FE01C56B41EA0541C4F88810C16BBF
S315080016E802EB41020468D4F8A010194041EA8201C5
S315080016F8C4F8A0100468D4F8A01021F4FE01056CFB
S3150800170841EA0541C4F8A010046C416C01FB0424A5
S315080017180268D2F8B010194041EA8401C2F8B0103C
S315080017280268D2F8B01021F4FE01856C41EA054139
S31508001738C2F8B010826CC16C01FB02440268D2F888
S31508001748AC10194041EA8401C2F8AC10026D416D2B
S3150800175801FB02420468D4F8F010194041EA8201F4
S31508001768C4F8F0100468D4F8F01021F47C11856DDB
S3150800177841EA0541C4F8F010816D02EB410204689C
S31508001788D4F8C0100B4043EA8202C4F8C0200268A5
S31508001798D2F8C03023F47C13C16D43EA0143C2F87A
S315080017A8C0300268D2F8C03023F07C53016E43EA91
S315080017B80163C2F8C030436B284A1A449200C266CD
S315080017C8836B02EB83030367C16B03EBC1034367B0
S315080017D8046C416C01FB04F103EB81038367846C99
S315080017E8C16C01FB04F103EB8103C367046D416D0A
S315080017F801FB04F103EB8103C0F88030816D03EB2C
S31508001808C103C0F88430C46D856E05FB04F403EB88
S315080018188403C0F88830016E01FB05F103EB8103E8
S31508001828C0F890300E498B4207D8D0F890309342CA
S315080018380ED9002342F8043BF7E7D0F89C3043F06A
S315080018482003C0F89C30032380F89830012000E074
S31508001858002030BC704700BF0300FFFF002B0010B4
S31508001868FCD30040F0B44C68002C2FD10E698C6864
S3150800187826430C6846EA84460D6ACC6944EA056438
S315080018888D692C434D692C43CD682C43D0F8847058
S31508001898806E03FB00F307EB830547F823606C604B
S315080018A808350020CB890E4CE35C834216D91418F8
S315080018B8E678A3781B0443EA0663647843EA0423B4
S315080018C8145C234345F8043B0430EBE70C698E683F
S315080018D826430C68264346F08046CDE7F0BC704799
S315080018E8385D00087047000030B595B004464C22AC
S315080018F8A04901A804F0C9F9002C00F0388123682A
S315080019089D4A934220D094F898300BB3226893697D
S3150800191823F01003936103F0C3FB054623689A690D
S3150800192812F0080F1AD003F0BBFB401B0A28F5D99A
S31508001938D4F89C3043F00103C4F89C30032384F898
S315080019489830012015B030BD03F580736360DAE777
S3150800195884F899302046FFF7C5FFD7E79A6942F019
S3150800196801029A6103F09CFB054623689A6912F0FE
S31508001978010F0FD103F094FB401B0A28F5D9D4F8B8
S315080019889C3043F00103C4F89C30032384F898304C
S315080019980120D7E79A6942F002029A61237C012B53
S315080019A840D02268936943F040039361637C012B16
S315080019B83ED02268936923F480439361A37C012B64
S315080019C83CD02268936943F48053936122689369EB
S315080019D823F44073A1680B4393612268936923F043
S315080019E8A40393612268136923F010031361E3685B
S315080019F8012B29D0002B2CD0022B00F09B802268C3
S31508001A08936943F0800393612268136943F01003CE
S31508001A181361E368032B1CD12268936943F02003FA
S31508001A28936116E02268936923F040039361BDE742
S31508001A382268936943F480439361BFE722689369F0
S31508001A4823F480539361C1E72268936943F004033A
S31508001A589361A3695A1EE369013B1B0243EA426381
S31508001A68226A013A13436269013A216843EA024342
S31508001A78CB61A368B3F5407F62D0236E33B1226881
S31508001A88D2F8C030616E0B43C2F8C030E36D226EDF
S31508001A98D3420DD02168D1F8C83023F00703A26EC7
S31508001AA814A800EB820252F84C2C1343C1F8C8302C
S31508001AB8236C6BB12168D1F8BC3023F00703626C3C
S31508001AC814A800EB820252F84C2C1343C1F8BC3018
S31508001AD8A36C73B12168D1F8BC3023F07003E26CAB
S31508001AE814A800EB820252F84C2C43EA0213C1F8F8
S31508001AF8BC30236D73B12168D1F8BC3023F4E06398
S31508001B08626D14A800EB820252F84C2C43EA0223B1
S31508001B18C1F8BC302268184B9A4222D00023C4F870
S31508001B289430C4F89C30012384F898302046FFF78F
S31508001B38ADFD07E72268936943F02003936188E7B8
S31508001B48A36A013BE26A013A43EA0223226B013A95
S31508001B5843EA0213626A013A216843EA0243CB6000
S31508001B688BE76268936823F003039360D6E701203E
S31508001B78E8E600BFC85C000800A0004090F8983066
S31508001B88013BDBB2012B07D9D0F89C3043F002039E
S31508001B98C0F89C3001207047CB680A68D2B9072B71
S31508001BA80ED08A68DB0643EA82730A6943EA024367
S31508001BB84A691343C26E496842F8213000207047C3
S31508001BC80A69CB691B0243EA02438A69134343F04D
S31508001BD86053EFE710B40A6942EA4372072B0ED03E
S31508001BE88C684B6943EA8473006F496800EBC10443
S31508001BF840F83120636000205DF8044B70478B6914
S31508001C08F2E710B490F89840E4B2012C09D0D0F85D
S31508001C189C3043F00403C0F89C3001205DF8044B5F
S31508001C287047920042EA011242EA43020168019BA0
S31508001C381A43C1F880200020F0E790F89830DBB204
S31508001C48012B07D0D0F89C3043F00403C0F89C3029
S31508001C5801207047022380F898300268936923F0B8
S31508001C68010393610023C0F89C301846704770B585
S31508001C7890F89840013CE4B2012C26D893FAA3F5CB
S31508001C88B5FA85F50668D6F8C040C4F30544A542F2
S31508001C980BD2D6F8CC401C420FD0D0F89C3043F073
S31508001CA84003C0F89C30012016E0D0F89C3043F079
S31508001CB82003C0F89C3001200EE093FAA3F3B3FA88
S31508001CC883F3FFF7CFFD002006E0D0F89C3043F0F9
S31508001CD80203C0F89C30012070BD90F89830DBB23A
S31508001CE8022B07D0D0F89C3043F00803C0F89C3084
S31508001CF8012070470368C3F8D01000207047000019
S31508001D08F0B490F89840E4B2022C40F0BA80402922
S31508001D180CD0412930D0046D8C4253D8D0F89C3069
S31508001D2843F02003C0F89C300120B1E00468D4F8D9
S31508001D38A05015F4FE0F0CD0D4F8A45015F07F0F58
S31508001D480FD1D0F89C3043F48073C0F89C3001203A
S31508001D589EE0D0F89C3043F02003C0F89C30012060
S31508001D6896E0D4F8A440C4F3052C446F456C0CFBE4
S31508001D7805F504EB85042DE00468D4F8B05015F48D
S31508001D88FE0F0CD0D4F8B45015F07F0F0FD1D0F849
S31508001D989C3043F48073C0F89C30012078E0D0F872
S31508001DA89C3043F02003C0F89C30012070E0D4F83A
S31508001DB8B440C4F3052C846FC56C0CFB05F504EB1D
S31508001DC8850407E0C46F456D01FB05F504EB85043A
S31508001DD84FF0000C256805F080455560002D2CD17C
S31508001DE82568C5F38A451560256805F00055956088
S31508001DF8256805F000451561A588D561656805F467
S31508001E087025D560656805F480155561656805F41B
S31508001E1800159561E57905F07F0515626568ED0F8A
S31508001E28556204F108050024D6891A4FBE5DA642F4
S31508001E3808D92E5D1E550134F6E7256825F0604554
S31508001E481560D1E740290AD041290DD01F290FD896
S31508001E580268012303FA01F1C2F8981002E0036840
S31508001E68C3F8A8C0002013E00368C3F8B8C0F9E7A8
S31508001E7801F01F010268012303FA01F1C2F89C1058
S31508001E88F0E7D0F89C3043F00803C0F89C300120EE
S31508001E98F0BC7047385D00080368D3F8CC300B42AD
S31508001EA801D00120704700207047402905D00368F3
S31508001EB8D3F8B40000F07F0070470368D3F8A4008D
S31508001EC800F07F007047000001F00303032B24D0BD
S31508001ED811F0010F0BD01D4BDA6822F03002DA60D8
S31508001EE8DA680243DA60DA6842F08802DA6011F0E2
S31508001EF8020F11D0154BD3F80C2122F03002C3F883
S31508001F080C21D3F80C211043C3F80C01D3F80C2183
S31508001F1842F08802C3F80C2170470C4BDA6822F0A5
S31508001F283002DA60D3F80C2122F03002C3F80C210B
S31508001F38DA680243DA60D3F80C211043C3F80C01B7
S31508001F489A6942F010029A61704700BF0020005251
S31508001F5830B411F0010F0BD0104DEB6823F4E6638B
S31508001F68EB60EC6842EA00231C4344F08404EC6006
S31508001F7811F0020F0FD00949D1F80C3123F4E663A2
S31508001F88C1F80C31D1F80C3142EA0022134343F068
S31508001F988403C1F80C3130BC704700BF00200052DA
S31508001FA8F8B5474B1B7D012B00F088800F46044681
S31508001FB8434B01221A7500229A61436813F0010FF0
S31508001FC80DD10026636813F0020F12D1CEB9236823
S31508001FD8012B1BD04FF0FF333B60A56859E0012160
S31508001FE84CF2503000F018FA06460028EAD00126C6
S31508001FF8E8E702214CF2503000F00EFA0028E5D046
S3150800200801262F4B00221A753046F8BD61682069EB
S31508002018FFF75AFF636813F0010F12D1636813F0CC
S31508002028020FEED002214CF2503000F0F5F900B15B
S315080020380126244AD2F80C3123F00803C2F80C31D9
S31508002048DFE701214CF2503000F0E6F900B101262D
S315080020581C4AD36823F00803D360DFE701214CF252
S31508002068503000F0D9F90646164AD168164B0B4087
S31508002078D3601CE002214CF2503000F0CDF9064638
S31508002088104AD2F80C11104B0B40C2F80C319EB905
S315080020980135E368A2681344AB42B2D9226961687C
S315080020A82846FFF755FF636813F0010FD6D1636812
S315080020B813F0020FEBD0DDE73D60A2E70226A3E79F
S315080020C8D012002000200052FBF8FFFF6A4B984206
S315080020D822D06A4B98422FD0694B98423CD0694B1C
S315080020E8984249D0684B984256D0684B984263D074
S315080020F8674B984270D0674B98427DD0664B98429A
S3150800210800F08A80654B984200F09680644B9842A6
S3150800211800F0A2800120704703F58843D3F8882089
S3150800212842F00102C3F88820D3F8882022F0010279
S31508002138C3F888200020704703F58043D3F8882021
S3150800214842F00202C3F88820D3F8882022F0020257
S31508002158C3F888200020704703F57053D3F8882001
S3150800216842F00402C3F88820D3F8882022F0040233
S31508002178C3F888200020704703F56053D3F88820F1
S3150800218842F00802C3F88820D3F8882022F008020B
S31508002198C3F888200020704703F55053D3F88820E1
S315080021A842F01002C3F88820D3F8882022F01002DB
S315080021B8C3F888200020704703F54053D3F88820D1
S315080021C842F02002C3F88820D3F8882022F020029B
S315080021D8C3F888200020704703F53053D3F88820C1
S315080021E842F04002C3F88820D3F8882022F040023B
S315080021F8C3F888200020704703F52053D3F88820B1
S3150800220842F08002C3F88820D3F8882022F080029A
S31508002218C3F888200020704703F51053D3F88820A0
S3150800222842F48072C3F88820D3F8882022F4807292
S31508002238C3F888200020704703F50053D3F8882090
S3150800224842F40072C3F88820D3F8882022F4007272
S31508002258C3F888200020704703F5E053D3F8882090
S3150800226842F48062C3F88820D3F8882022F4806272
S31508002278C3F8882000207047000002580004025856
S3150800228800080258000C0258001002580014025898
S3150800229800180258001C0258002002580024025848
S315080022A800280258F0B40C6894FAA4F4B4FA84F432
S315080022B82BE08E68826803FB03F505EB450722EADF
S315080022C8070205FB06F52A4382600E68CD68426850
S315080022D822EA060205FB06F52A4342600F69C66824
S315080022E803FB03F505EB4502D243164005FB07F742
S315080022F83E43C6604E68022E14D04B6806683240C4
S3150800230805FB03F31343036001340B6833FA04F23D
S315080023182BD00122A2401340F6D04A68013A012A76
S31508002328DCD8C6E7FF2B0ED8066A05FB03F707FBBA
S3150800233803F3C3EB031726EA07074E6903FB06F3FD
S315080023483B430362D9E7466A1B0A03FB03F707FB05
S3150800235803F707FB03F3C3EB031726EA07074E69D8
S3150800236803FB06F33B434362C7E70020F0BC70470C
S31508002378024AD36843F08073D3607047004802580E
S31508002388144BDB6813F0010F09D0124B124A5A6036
S3150800239802F188325A60DB6813F0010F14D10D4B2D
S315080023A8D3F80C3113F0010F10D00A4B0A4AC3F8B8
S315080023B8042102F18832C3F80421D3F80C3113F04A
S315080023C8010F05D10020704701207047002070478B
S315080023D80120704700200052230167450D4BDA6833
S315080023E842F00102DA60DB6813F0010F0DD0094BE1
S315080023F8D3F80C2142F00102C3F80C21D3F80C31AA
S3150800240813F0010F03D00020704701207047012000
S31508002418704700BF00200052F8B505460E4602F080
S315080024283FFE0746012E09D0364C17E002F038FE63
S31508002438C01BA84260D88DB903204EE004240DE0DD
S31508002448314BD3F8103124EA030333F000430CBFA9
S31508002458012300236BB1B5F1FF3FE7D134F004033C
S31508002468EED1294B1B6934EA03030CBF0123002369
S31508002478F0E7012E1CD0244BD3F8103123F068431B
S3150800248823F480135B0C5B0443F0004333F00242E9
S3150800249817D1012E25D01C4BD3F8103113F4803FE1
S315080024A82ED0194B4FF48032C3F81421002014E0BB
S315080024B8154B1B6923F0684323F480135B0C5B04F4
S315080024C8E4E712498A691A438A61002B06DA23F077
S315080024D800430D4AC2F814310120F8BD0A4A53616F
S315080024E8FAE7094B1B6913F4803F07D0064B4FF4EC
S315080024F880325A610020F0E70320EEE70020ECE777
S315080025080020EAE70400008000200052D0120020CC
S315080025182C4B1B7D012B51D070B50C461546294B03
S3150800252801221A7501F17841B1F5801F38D216468D
S31508002538244B00229A6131464CF25030FFF76CFF63
S31508002548034640BB012E2DD01F4AD2F80C3143F062
S315080025580203C2F80C31BFF36F8FBFF34F8F0823FE
S3150800256855F8042B44F8042B013B13F0FF03F7D165
S31508002578BFF36F8FBFF34F8F31464CF25030FFF7DA
S315080025884BFF0346012E13D00F49D1F80C2122F030
S315080025980202C1F80C210B4A00211175184670BDB4
S315080025A80226C5E7084AD36843F00203D360D2E790
S315080025B80549CA6822F00202CA60ECE702231846EF
S315080025C8704700BFD01200200020005200230133B4
S315080025D80C4A934211D80269002AF8DA036943F0CB
S315080025E80103036100230133064A934207D80269A7
S315080025F812F0010FF7D10020704703207047032017
S31508002608704700BF400D030084B010B5044603A800
S3150800261880E80E00089B012B1DD1A36B23F4803399
S31508002628A363E2681A4B1340E360E36823F4401394
S31508002638E3600F9B012B09D02046FFF7C7FF069BCF
S31508002648012B1BD0BDE8104004B07047E36843F47B
S315080026588013E360F0E7E36843F04003E36020464D
S31508002668FFF7B4FF0C9B23B9A36B43F48033A3632A
S31508002678E5E7A36B23F48033A363E0E7A36843F095
S315080026880603A360A36843F02003A360DAE700BF44
S31508002698BFFFBDFF022A0AD00921C26822F4705278
S315080026A8C260C36843EA8123C36000207047274B8A
S315080026B80B44274A934237D9264B0B44264A93425A
S315080026C834D9264B0B44264A934231D9254B0B4419
S315080026D802F5C332A03293422CD9234B0B44234A22
S315080026E8934229D9224B0B4402F5922202F57872B5
S315080026F8934223D91F4B0B4402F5C32202F52072D5
S3150800270893421DD91C4B0B4402F5B71202F55872B1
S31508002718934217D9194B0B4402F5122202F5F862AF
S31508002728934211D80721B8E70F21B6E70E21B4E777
S315080027380D21B2E70C21B0E70B21AEE70A21ACE779
S315080027480921AAE70821A8E70621A6E7405327FF93
S31508002758FF340C00401E1BFF3F420F0000DC0BFF36
S315080027687F4F1200808CF9FE60B6E5FE5FE316001F
S3150800277800D3CEFEC05BB3FE00CA91FEE05459FEF4
S31508002788836843F00103836000207047836823F059
S31508002798010383600020704708B5C36823F0C04367
S315080027A8C360012909D069B9C36843F08043C36087
S315080027B83220FEF731FC002008BDC36843F00053F9
S315080027C8C360F5E70120F7E7890141F020010161B7
S315080027D800230133054A934205D8026912F0200FEF
S315080027E8F7D1002070470320704700BF400D03004B
S315080027F81023036100230133054A934205D8026969
S3150800280812F0100FF7D1002070470320704700BF59
S31508002818400D0300D0F800381943C0F80018002006
S315080028287047000084B0F8B5044607A880E80E008B
S31508002838254600230E2B07D803F1400204EB820233
S31508002848002151600133F5E7119B23BBD4F80438FE
S3150800285843F00203C4F80438A36B23F40013A363F4
S31508002868236843F040032360236843F0800323600A
S315080028780023C4F8003E04F50066D4F80038C4F806
S3150800288800380C9B012B10D1099B4BB90021204617
S31508002898FFF7C0FF0DE0A36B43F40013A363E7E754
S315080028A801212046FFF7B6FF03E003212046FFF77C
S315080028B8B1FF10212046FFF787FF074600B1012719
S315080028C82046FFF795FF00B101270023336173619E
S315080028D8F3610AE0C3B94FF00060C2F800090022A4
S315080028E80A614FF67F328A600133079A9A4210D9ED
S315080028F805EB431202F51061D2F800090028E9DB56
S315080029080020C2F80009EAE74FF09040C2F800092B
S31508002918E5E700230AE0C3B94FF00060C2F8000BE8
S3150800292800220A614FF67F328A600133079A9A4273
S3150800293810D905EB431202F53061D2F8000B0028CE
S31508002948E9DB0020C2F8000BEAE74FF09040C2F82E
S31508002958000BE5E7336923F4807333610023A36129
S315080029686FF0804363610A9B1BB9A36943F01003A0
S31508002978A361A2690A4B1343A3610D9B1BB1A36903
S3150800298843F00803A361119B012B04D03846BDE820
S31508002998F84004B07047A269024B1343A361F5E7F0
S315080029A800383C8004000040D0F8083813F00603C5
S315080029B805D0062B18BF022B03D10220704700202A
S315080029C870470F207047000070B40B784A78012AC0
S315080029D820D0D0F81C2803F00F060124B44042EA98
S315080029E80442C0F81C2800EB4310D0F8003B13F447
S315080029F8004F0CD1D0F8002B8B68C3F30A03C978AB
S31508002A0843EA81431343134A1A43C0F8002B0020AC
S31508002A1870BC7047D0F81C4803F00F06B24092B253
S31508002A282243C0F81C2800EB4310D0F8002912F4FA
S31508002A38004FECD1D0F800498A68C2F30A02C9786F
S31508002A4842EA814242EA8353234302491943C0F8BA
S31508002A580019DCE70080001070B40B784A78012A60
S31508002A681FD0D0F83C5803F00F06012404FA06F6DE
S31508002A7825EA0645C0F83C58D0F81C58097801F0EC
S31508002A880F018C4025EA0444C0F81C4800EB4310A3
S31508002A98D0F8002B124B1340C0F8003B002070BC3E
S31508002AA87047D0F83C6803F00F0402FA04F4A4B29D
S31508002AB826EA0404C0F83C48D0F81C48097801F00E
S31508002AC80F018A4092B224EA0202C0F81C2800EBD9
S31508002AD84310D0F80039034A1A40C0F80029DDE740
S31508002AE80078F3EF007833EC70B40B784C78012C47
S31508002AF824D000EB431000F530631D693E4C2C408A
S31508002B081C611D693D4C2C401C614C690CB18C68D4
S31508002B184C611C6944F400241C611C698D68C5F362
S31508002B2812052C431C61012A61D0D0F8003B43F0FA
S31508002B380443C0F8003B002070BC70474C695CBB76
S31508002B4800EB4314D4F810692C4D3540C4F81059D5
S31508002B58D4F8105945F40025C4F81059D4F8106962
S31508002B68254D3540C4F81059012A31D000EB4313D6
S31508002B78D3F8002942F00442C3F800294B69002B10
S31508002B88D9D0D0F83428097801F00F040121A140DA
S31508002B980A43C0F83428CEE700EB431404F510645A
S31508002BA82669154D354025612669144D3540256138
S31508002BB84E698D68AE4200D94D61256945F40025F0
S31508002BC8256125694E69C6F3120635432561CBE7A3
S31508002BD80A691AB100EB4311C1F8142900EB43102E
S31508002BE8D0F8002942F00442C0F80029A3E7CA68C9
S31508002BF8002A9AD05A6198E70000F8FFFFFF07E015
S31508002C0870B49DF80C4064B903339E08B44208D2E0
S31508002C1800EB023303F5805351F8045B1D60013459
S31508002C28F4E7002070BC7047F0B583B00B784C7891
S31508002C38012C29D000EB431303F5306426697C4D33
S31508002C483540256126697B4D354025614D69002D3E
S31508002C5840F0BF8025698E68C6F31206354325619C
S31508002C68256945F400252561012A00F0C780CA7838
S31508002C78012A00F0C980D3F8002B42F00442C3F8B1
S31508002C88002B002003B0F0BD4C6974BB00EB43145D
S31508002C98D4F81069674D3540C4F81059D4F8105956
S31508002CA845F40025C4F81059D4F81069604D354024
S31508002CB8C4F81059012A4AD000EB4313D3F800493F
S31508002CC844F00444C3F80049CC78012C68D04B6911
S31508002CD8002BD6D0D0F83428097801F00F04012142
S31508002CE8A1400A43C0F83428CBE700EB4314D4F8CC
S31508002CF810694F4D3540C4F81059D4F810694D4D30
S31508002D083540C4F81059D4F810694D698F683D44A0
S31508002D18013DB5FBF7F5484F07EAC5453543C4F8FD
S31508002D281059D4F810594E69C6F312063543C4F833
S31508002D38105904F51064CD78012DBBD1256925F005
S31508002D48C0452561256945F000552561B2E70A6938
S31508002D581AB100EB4314C4F81429CA78012A08D012
S31508002D6800EB4313D3F8002942F00442C3F80029BC
S31508002D7887E7D0F8082812F4807F08D100EB4311BA
S31508002D88D1F8002942F00052C1F80029E8E700EB1B
S31508002D984311D1F8002942F08052C1F80029DFE72B
S31508002DA8D0F8084814F4807F0CD1D3F8004944F0C9
S31508002DB80054C3F8004900928B8A0A78C968FFF755
S31508002DC81FFF5EE7D3F8004944F08054C3F800496A
S31508002DD8F1E78E683544013DB5FBF6F52669164FC9
S31508002DE807EAC5473E43266127698E68ADB206FBE2
S31508002DF805F5C5F312053D43256135E7CA68002A76
S31508002E083FF435AF626132E7D0F8082812F4807FBC
S31508002E1806D1D3F8002B42F00052C3F8002B2AE754
S31508002E28D3F8002B42F08052C3F8002B23E700BFE3
S31508002E380000F8FFFFFF07E00000F81F03329208BA
S31508002E48002393420CD210B400F58054246841F844
S31508002E58044B01339342F7D308465DF8044B704791
S31508002E68084670470B784A78012A14D000EB4310B5
S31508002E78D0F8002B002A06DB2BB1D0F8003B23F04C
S31508002E888043C0F8003BD0F8003B43F40013C0F871
S31508002E98003B0020704700EB4310D0F80029002AB1
S31508002EA806DB2BB1D0F8003923F08043C0F8003987
S31508002EB8D0F8003943F40013C0F80039E9E70B786D
S31508002EC84A78012A0ED000EB4310D0F8003B23F4C9
S31508002ED80013C0F8003BCB78023BDBB2012B15D9AF
S31508002EE80020704700EB4310D0F8003923F400138C
S31508002EF8C0F80039CB78023BDBB2012BF0D8D0F802
S31508002F08003943F08053C0F80039E9E7D0F8003BA8
S31508002F1843F08053C0F8003BE2E738B50546044657
S31508002F2800220E2A09D804EB42134FF67F31C3F85C
S31508002F380819C3F8081B0132F3E70022C5F8102858
S31508002F48C5F81428C5F81C282846FFF751FC034677
S31508002F5808B1184638BD10212846FFF735FC034640
S31508002F68F7E7D0F8003823F4FE63C0F80038D0F83D
S31508002F780038090101F4FE610B43C0F80038002047
S31508002F88704708B5D0F8043823F00203C0F80438A7
S31508002F980320FEF741F8002008BD08B5D0F8043824
S31508002FA843F00203C0F804380320FEF735F800207A
S31508002FB808BD4269806910407047D0F8183800F58E
S31508002FC80060C0691840000C7047D0F8183800F53A
S31508002FD80060C069184080B2704700EB4111D1F80B
S31508002FE8082B00F5006040691040704710B4D0F807
S31508002FF81048D0F8343801F00F02D340DB01DBB2B1
S31508003008234300EB411000F51060806818405DF80E
S31508003018044B7047406900F001007047D0F8002952
S31508003028054B1340C0F80039D0F8043843F48073C8
S31508003038C0F804380020704700F8FFFF10B4046C85
S31508003048154B9C4203D9D0F8003B002B16DB00240D
S31508003058C0F8104BD0F8104B44F40024C0F8104BB5
S31508003068D0F8104B44F01804C0F8104BD0F8104BA1
S3150800307844F0C044C0F8104B012903D000205DF87D
S31508003088044B7047C0F8142BD0F8003B43F0802354
S31508003098C0F8003BF2E700BF0A30544F724B1B6971
S315080030A803F03803102B00F0DB80182B10D00BB177
S315080030B86E4870476C4B1B6813F0200F00F0D280DF
S315080030C8694B1868C0F3C100694B23FA00F07047CA
S315080030D8654A916A01F00301906AC0F30510D36A3C
S315080030E803F00103526BC2F3CC0203FB02F307EEAB
S315080030F8903AF8EE677A002800F0B580012966D07C
S31508003108F9B1022900F08F8007EE100AF8EE476A2F
S315080031189FED586A86EE267A534B1B6BC3F3080352
S3150800312806EE903AF8EE666A9FED536A67EE867A77
S3150800313876EEA77AF7EE006A77EEA67A27EE277A6A
S3150800314861E0494B1B6813F0200F23D046490A68EB
S31508003158C2F3C102464BD34007EE103AF8EE476A67
S3150800316807EE100AB8EE476A86EE867A0B6BC3F343
S31508003178080306EE903AF8EE666A9FED3F6A67EE30
S31508003188867A76EEA77AF7EE006A77EEA67A27EEBB
S31508003198277A38E007EE100AF8EE476A9FED376A8D
S315080031A886EE267A304B1B6BC3F3080306EE903A75
S315080031B8F8EE666A9FED306A67EE867A76EEA77A43
S315080031C8F7EE006A77EEA67A27EE277A1BE007EE6F
S315080031D8100AF8EE476A9FED276A86EE267A224B8A
S315080031E81B6BC3F3080306EE903AF8EE666A9FED82
S315080031F8226A67EE867A76EEA77AF7EE006A77EE9F
S31508003208A67A27EE277A184B1B6BC3F34623013396
S3150800321807EE903AF8EE677AC7EE276AFCEEE67A82
S3150800322817EE900A704707EE100AF8EE476A9FED00
S31508003238146A86EE267A0C4B1B6BC3F3080306EE54
S31508003248903AF8EE666A9FED0C6A67EE867A76EE2D
S31508003258A77AF7EE006A77EEA67A27EE277AD2E7F4
S3150800326808487047024870470044025800093D005C
S315080032780090D0030024744A000000390024744CD6
S315080032880024F44A00127A0008B5FFF707FF0B4A2C
S315080032989369C3F303230A49CB5C03F01F0320FA97
S315080032A803F3926902F00F02885C00F01F0023FA04
S315080032B800F0044A1060044A136008BD0044025826
S315080032C8185D0008300400202C040020014B186003
S315080032D8704700BF2C04002038B5036813F0010FA7
S315080032E840F08C800D4604460368454A1A408B68A8
S315080032F809690B4369690B43E9690B43134303607F
S31508003308EB68426822F4405213434360AB6982680B
S3150800331822F44072134383603A4B984216D03A4BCC
S3150800332898421CD0394B98421DD0394B98421ED02A
S31508003338384B98421FD0384B984220D0374B984282
S3150800334821D0374B984222D001204EE03548FEF767
S31508003358E9F8002848D06A68EAB9012045E0324801
S31508003368FEF7E0F8F5E73048FEF7DCF8F1E72E480F
S31508003378FEF7D8F8EDE72C48FEF7D4F8E9E7294828
S31508003388FEF7D0F8E5E72848FEF7CCF8E1E726483F
S31508003398FEF7C8F8DDE72B68E9690B2B2CD8B1F5D9
S315080033A8004F0DD0DBB2214951F82330B0FBF3F3B7
S315080033B803EB5203B3FBF2F39BB2E360002014E07D
S315080033C8DBB21A4951F82330B0FBF3F0530803EB84
S315080033D84000B0FBF2F34FF6F0721A40C3F342030B
S315080033E81343E360002000E00120E26A22F00F029E
S315080033F82B881343E36202E00020F6E7012038BD74
S31508003408F369FFEF001001400044004000480040FF
S31508003418004C00400050004000140140007800406D
S31508003428007C00400803000708000007485D0008FC
S315080034380649CB6823F4E0631B041B0C000200F45E
S31508003448E0600343024A1A43CA60704700ED00E089
S315080034580000FA0530B4154BDB68C3F30223C3F141
S315080034680704042C28BF04241D1D062D01D9033B77
S3150800347800E000234FF0FF3505FA04F421EA0401B9
S31508003488994005FA03F322EA03031943002805DBE2
S315080034980901C9B2064B195430BC704700F00F0031
S315080034A80901C9B2034B1954F6E700BF00ED00E05D
S315080034B800E400E014ED00E00138B0F1807F0AD29C
S315080034C8064B5860064AF02182F8231000209860B7
S315080034D807221A6070470120704700BF10E000E015
S315080034E800ED00E030B40468606A29B940EA024091
S315080034F8A062002030BC70470D46A36A00EB134053
S315080035080023691E8B4209D203F1400104EB8101AD
S31508003518496800EB11400133DBB2F2E740EA0240A2
S3150800352805F13F0104EB81014860E2E70368596247
S3150800353800207047024603680121C0F8FC130020E2
S3150800354882F8F4039A6942F000629A61596D024A50
S315080035580A435A65704700BF0300001070472DE9F3
S31508003568F04782B0D0F80080CA00521A9300034484
S315080035785A6D1B6D9A4255D8C1469B1AC1EBC104B0
S31508003588A2000244526C9A4200D31A460C460746D1
S3150800359802F1030A4FEA9A0A15E006F1030A4FEA06
S315080035A89A0AE3001B1B9D003D44A96C3B7C0093CB
S315080035B8B3B2E2B24046FFF723FBAB6C3344AB64C5
S315080035C86B6D1E446E6509EB441303F510639B691E
S315080035D89BB2534512D3E3001B1B9A003A44516D1C
S315080035E8136D99420AD24BB15B1AC4EBC4018A001F
S315080035F83A44566C9E42D0D31E46CEE7E3001B1BC0
S31508003608980007443A6D7B6D9A420FD804F00F0468
S315080036180123A340D8F8344824EA0304C8F83448F0
S31508003628002000E0012002B0BDE8F0870020FAE794
S315080036387047F0B58BB0002800F0918004460568FD
S3150800364890F8BD3323B3032384F8BD33EB6B13F427
S31508003658807F01D1002323612068FFF797F8254664
S3150800366855F8107B6E460FCD0FC60FCD0FC695E8D9
S31508003678030086E80300231D0ECB3846FEF7C4FF71
S3150800368858B1022384F8BD33012528460BB0F0BD8E
S3150800369880F8BC33FFF7CCFFD5E700212068FFF791
S315080036A87BF800236568AB4216D2D900C81A82008F
S315080036B82244012082F83D0082F83C30A2F84230C4
S315080036C8002082F83F0050649064CA1A9100214489
S315080036D808650133DBB2E5E700239D4216D9D80011
S315080036E8C11A8A002244002182F8FD1182F8FC31A9
S315080036F882F8FF11C2F80412C2F80812C21A90001A
S315080037082044C0F810120133DBB2E6E7254655F81F
S31508003718107B6E460FCD0FC60FCD0FC695E8030072
S3150800372886E80300231D0ECB3846FFF77BF80546C7
S3150800373860B9002384F83830012384F8BD33636AF6
S31508003748012B08D02068FFF728FC9EE7022384F897
S31508003758BD33012599E72046FFF7ECFEF2E7012578
S3150800376893E77047026890F8BC33012B19D010B557
S31508003778012380F8BC33836A012B0AD00446006803
S31508003788FFF7FFFB2068FEF7FBFF002084F8BC0361
S3150800379810BD8369012BF1D0936B43F4803393638F
S315080037A8ECE70220704738B590F8BC33012B18D0DF
S315080037B80446012380F8BC330068FEF7E7FF206853
S315080037C8FFF7ABFB054628B1002384F8BC3301256F
S315080037D8284638BD2068FFF7E0FB002384F8BC3389
S315080037E8F6E70225F4E768B110B50446032380F81E
S315080037F8BD33FFF7D8FF2046FFF7B3FF002084F84C
S31508003808BD0310BD0120704770B504460D46006813
S31508003818066C00EB411303F530639A6821690129A0
S3150800382811D037498E4254D03DB9C5EBC50293002D
S315080038382344D3F81032002B5CD0E9B2204600F0B6
S31508003848C1FF002070BD12F0080F09D02D498E421D
S31508003858F7D912F4004FF4D04FF400429A60F0E713
S3150800386812F0200F02D020229A60EAE712F0280FF9
S31508003878E7D124498E4206D912F4004F03D04FF4F3
S3150800388800429A60DDE7E900491B8A002244D2F81B
S3150800389804121B69C3F31203C91AC2F81412D2F820
S315080038A80412D2F808320B44C2F8083235B9C5EB07
S315080038B8C50293002344D3F8103223B1E9B220464F
S315080038C800F080FFBDE704F571720121FFF7B6FB2A
S315080038D8F4E712F4004F03D04FF400429A60B0E7B9
S315080038E812F0200F01D020229A60E9B2204600F093
S315080038F869FFA6E704F571720021FFF79FFB9CE7AD
S315080039080A31544F0A30544F38B5044603681D6CBB
S3150800391803EB4111D1F8082B0E4B9D4207D901F547
S31508003928306112F4004F02D04FF400438B602046F2
S3150800393800F040FF074B9D4202D92369012B01D0AD
S31508003948002038BD04F5717201212068FFF776FB5F
S31508003958F6E700BF0A30544F2DE9F84F04460568C4
S315080039682846FFF757FB08B1BDE8F88F2F460646E5
S315080039782068FFF71EFB0028F6D02068FFF719FB1A
S3150800398810F0020F04D02268536903F0020353614A
S315080039982068FFF70EFB10F0100F15D02268936900
S315080039A823F010039361D5F8208008F00F09C8F3AF
S315080039B84343022B00F08580062B00F0A580226879
S315080039C8936943F0100393612068FFF7F2FA10F43D
S315080039D8002F40F0AD802068FFF7EBFA10F4802F2F
S315080039E840F0F1802068FFF7E4FA0028C0F25F810A
S315080039F82068FFF7DEFA10F4006F0AD0D5F8083801
S31508003A0813F0010F40F06D812268536903F40063CF
S31508003A1853612068FFF7CDFA10F0006F15D02268B9
S31508003A28536903F00063536194F8F433002B40F0AC
S31508003A385C81012184F8F41323685B6DC3F383035F
S31508003A48C4F8F8332046FFF789FD2068FFF7B1FA6E
S31508003A5810F4805F40F04D812068FFF7AAFA10F449
S31508003A68005F40F0AB812068FFF7A3FA10F0080F53
S31508003A7840F0BC812068FFF79CFA10F4801F40F0DC
S31508003A88BE812068FFF795FA10F4001F40F0C1813F
S31508003A982068FFF78EFA10F0804F40F0C48120683E
S31508003AA8FFF787FA10F0040F3FF45EAF23685D68E6
S31508003AB815F0040F40F0C081226853682B43536001
S31508003AC852E747F6F07318EA030F3FF478AF4FEA60
S31508003AD818184FEAC90BABEB09034FEA830AA24445
S31508003AE8C8F30A02DAF808122846FFF7A7F9C8F34E
S31508003AF80A08DAF808324344CAF80832DAF81432F7
S31508003B084344CAF814325AE7082204F5717128465C
S31508003B18FFF794F9C8F30A184FEAC903A3EB090192
S31508003B288A002244D2F814324344C2F8143246E7CB
S31508003B382068FFF742FA8046B14617E007EB4913B3
S31508003B480122C3F8082B49462046FFF75DFE1DE00B
S31508003B5807EB49130822C3F8082B49462046FFF7FE
S31508003B68D3FE16E009F101094FEA5808B8F1000F23
S31508003B783FF431AF18F0010FF4D05FFA89F12068E5
S31508003B88FFF72BFA824610F0010FD7D11AF0080F63
S31508003B98DED11AF0100F04D007EB49131022C3F828
S31508003BA8082B1AF0200F04D007EB49132022C3F874
S31508003BB8082B1AF4005FD5D007EB49134FF40052C7
S31508003BC8C3F8082BCEE72068FFF7FFF98046B14609
S31508003BD82AE05946204600F001FE1AF0080F04D0DC
S31508003BE807EB49130822C3F808291AF0100F04D05E
S31508003BF807EB49131022C3F808291AF0400F04D016
S31508003C0807EB49134022C3F808291AF0020F04D013
S31508003C1807EB49130222C3F808291AF0800F41D185
S31508003C2809F101094FEA5808B8F1000F3FF4DAAE6E
S31508003C3818F0010FF4D05FFA89FB59462068FFF798
S31508003C48D5F9824610F0010FC7D009F00F030121F4
S31508003C5801FA03F2D7F8343823EA0203C7F83438E6
S31508003C6807EB4913C3F8081923698B42B1D14FEA00
S31508003C78C902A2EB090293002344596C9A6C0A44B8
S31508003C889A64B9F1000FA4D1C9EBC9029300234479
S31508003C981B6D002B9DD104F5717201212068FFF771
S31508003CA8CDF996E749462046FFF759FCB8E7D5F80F
S31508003CB8043823F00103C5F8043894F8F433012BC3
S31508003CC808D0204600F0D0FD2268536903F0004367
S31508003CD853618DE6002184F8F4132046FFF73EFC6D
S31508003CE8F2E7204600F0A6FD8EE6204600F0A2FD83
S31508003CF8ABE605F50068D8F8043023F00103C8F8E0
S31508003D08043010212068FEF75FFD20E007EB461314
S31508003D184FF67F31C3F80819D3F8002922F40012A0
S31508003D28C3F80029D3F8002942F00062C3F800292D
S31508003D38C3F8081BD3F8002B22F40012C3F8002B8B
S31508003D48D3F8002B42F00062C3F8002B01366368EB
S31508003D58B342DBD8D8F81C3043F00113C8F81C3036
S31508003D68236BEBB1D8F8843043F00B03C8F88430DA
S31508003D78D8F8443043F00B03C8F84430D5F800386F
S31508003D8823F4FE63C5F8003804F57172217C2068AF
S31508003D98FFF754F92268536903F4805353615BE6C5
S31508003DA8D8F8142042F22B031343C8F81430D8F86D
S31508003DB8103043F00B03C8F81030DFE72068FFF728
S31508003DC82DF92068FEF7F0FDE0602568FFF75CFA34
S31508003DD8227B01462846FEF75DFC204600F010FDCA
S31508003DE82268536903F4005353613CE6204600F001
S31508003DF800FD2268536903F0080353613AE6002177
S31508003E08204600F040FD2268536903F48013536185
S31508003E1837E60021204600F030FD2268536903F48E
S31508003E280013536134E6204600F033FD22685369CF
S31508003E3803F08043536132E6204600F034FD3BE642
S31508003E48026890F8BC33012B16D010B5012380F808
S31508003E58BC33836A012B07D004460068FFF791F83C
S31508003E68002084F8BC0310BD8369012BF4D0936B3A
S31508003E7843F480339363EFE70220704790F8BC3326
S31508003E88012B0BD010B50446012380F8BC33006813
S31508003E98FFF783F8002084F8BC0310BD022070479A
S31508003EA890F8BC33012B0DD010B50446012380F8D1
S31508003EB8BC3380F838100068FFF753F8002084F8F8
S31508003EC8BC0310BD02207047F8B511F0800F27D142
S31508003ED801F00F05EE00771BBC00274604F5FC74B5
S31508003EE8044404340744002587F8FD5101F00F01FE
S31508003EF82170A260E370627802B1E180022B1ED0BD
S31508003F0890F8BC33012B1DD00546012380F8BC3335
S31508003F1821460068FEF758FD002085F8BC03F8BD61
S31508003F2801F00F06F500AF1BBC00274638340444D9
S31508003F3804343E460644012586F83D50D6E7002354
S31508003F482371DDE70220EAE738B511F0800F20D1A2
S31508003F5801F00F04E200151BAB001D4603F5FC73C0
S31508003F68034404330544002285F8FD2101F00F01B6
S31508003F78197090F8BC23012A1AD00446012280F841
S31508003F88BC2319460068FEF767FD002084F8BC03C1
S31508003F9838BD01F00F04E200151BAB001D46383387
S31508003FA8034404332C460444012284F83D20DDE703
S31508003FB80220EDE770B501F00F05EE00711B8C00C5
S31508003FC804F5FC740444211D761BB4000444C4F8A3
S31508003FD80822C4F810320023C4F8143284F8FD31D4
S31508003FE884F8FC510369012B06D065B9DAB2006872
S31508003FF8FEF77AFD002070BDC5EBC506B40004447B
S31508004008C4F80C22F1E7DAB20068FEF70DFEF1E70C
S3150800401801F00F01C1EBC1018B001844D0F8140256
S31508004028704770B501F00F05EE00711B8C00383427
S315080040380444211D761BB4000444A26423650023A6
S315080040486365012384F83D3084F83C500369012BE5
S3150800405806D05DB9DAB20068FEF746FD002070BDE5
S31508004068C5EBC506B4000444E264F2E7DAB20068B0
S31508004078FEF7DAFDF2E738B501F00F0543689D4209
S3150800408836D811F0800F20D1CA00541AA3001C464E
S3150800409803F5FC730344043322460244002182F8DC
S315080040A8FD1101229A701D7090F8BC23012A21D0AF
S315080040B80446012280F8BC2319460068FEF7D2FE9A
S315080040C87DB1002084F8BC0338BDEA00511B8B007B
S315080040D819463833034404330144012281F83D2044
S315080040E8DFE704F57172217C2068FEF7A7FFE8E789
S315080040F80120E9E70220E7E710B501F00F04436855
S315080041089C422CD811F0800F1DD1E3001A1B910090
S315080041180A4601F5FC71014404310244002382F879
S31508004128FD3100238B700C7090F8BC33012B18D026
S315080041380446012380F8BC330068FEF7C0FE002059
S3150800414884F8BC0310BDE3001A1B91000A463831EF
S31508004158014404310244012382F83D30E1E7012095
S31508004168F0E70220EEE7000012230B8000487047AC
S315080041785804002004230B80004870476C0400206C
S315080041880023934216D230B40BE0373401F81340B3
S3150800419800015C00013400250D550133DBB293425A
S315080041A806D2040F092CF0D8303401F81340EFE78B
S315080041B830BC70477047000038B50A4B1868043396
S315080041C81C6804331B68C01800D138BD064D082280
S315080041D8A91CFFF7D5FF042205F112012046FFF7AF
S315080041E8CFFFF2E700E8F11F7004002008B51A238C
S315080041F80B80FFF7E1FF014808BD00BF70040020E7
S3150800420808B50A4628B905490548FCF79AFC03483B
S3150800421808BD02490248FCF794FCF8E7EC120020AE
S31508004228A85D000810B5044C0A4621460348FCF761
S3150800423888FC204610BD00BFEC120020985D0008D7
S3150800424808B50A4628B905490548FCF77AFC03481B
S3150800425808BD02490248FCF774FCF8E7EC1200208E
S31508004268785D000808B50A4628B905490548FCF7DF
S3150800427868FC034808BD02490248FCF762FCF8E7EF
S31508004288EC120020805D0008014B1880704700BFBB
S315080042980E05002008B500F0FBFE0E4B1B68984279
S315080042A80FD30D4B1B786BB90B4B01221A700B4BAE
S315080042B880229A6100F0ECFE094B1B881844054BCE
S315080042C8186008BD044B00221A70044B4FF400020C
S315080042D89A61EFE71405002010050020000402582B
S315080042E80E050020024B4FF400029A61704700BF82
S315080042F80004025808B5054B1B6913F4005F03D17F
S31508004308FFF7F0FF012008BD0020FCE70008025867
S3150800431808B56420FFF7B8FF08BD08B5FFF7BAFF68
S3150800432808BD70477047704708B5574A136823F0A1
S315080043380F0343F004031360136803F00F03042BF9
S3150800434840F09C80514AD36823F0070343F00203E0
S31508004358D360936943F4404393614D4B1A6842F41A
S3150800436880221A601A6842F480321A60484B1B6821
S3150800437813F4003FFAD0464B9A6A22F0030242F039
S3150800438802029A62DA6A42F48032DA62DA6A42F435
S315080043980032DA62DA6A22F00C0242F00402DA62C1
S315080043A8DA6A22F00202DA629A6A22F47C7242F027
S315080043B840029A621A6B3749114040F2DF120A43E3
S315080043C81A631A6B22F47E4242F400721A631A6B55
S315080043D822F4FE0242F498121A631A6B22F0FE427D
S315080043E842F080721A631A6842F080721A60284B83
S315080043F81B6813F0007FFAD0254B9A6922F00F0242
S3150800440842F008029A611A6922F0070242F003028A
S315080044181A619A6922F470629A619A6922F00F02FF
S3150800442842F008029A61DA6922F0700242F0400204
S31508004438DA61DA6922F4E06242F48062DA619A693A
S3150800444822F0700242F040029A611A6A22F070025B
S3150800445842F040021A6210490A6822F007020A6006
S315080044681A6D22F040521A655A6D22F4401242F427
S3150800447880125A650948FEF729FF08BD67210848CA
S3150800448800F0D4FA5EE700BF002000520048025840
S315080044980044025800FEFFFF5444025800389C1C8A
S315080044A8BC5D000808B5FCF789FDFFF73DFF08BDA8
S315080044B808B5FFF7F7FF00F0C5FA00F0D1FAFCE7F0
S315080044C82DE9F0418EB0514CD4F8F43043F002038C
S315080044D8C4F8F430D4F8F43003F002030793079BC2
S315080044E8D4F8E03043F00103C4F8E030D4F8E030FB
S315080044F803F001030693069BD4F8E03043F0020361
S31508004508C4F8E030D4F8E03003F002030593059BBD
S31508004518D4F8E03043F00403C4F8E030D4F8E030C7
S3150800452803F004030493049BD4F8E03043F008032B
S31508004538C4F8E030D4F8E03003F008030393039B8B
S31508004548D4F8E83043F48023C4F8E830D4F8E830DF
S3150800455803F480230293029BD4F8EC3043F4807367
S31508004568C4F8EC30D4F8EC3003F480730193019B5B
S31508004578802308930123099300250A950B950C9522
S31508004588234F08A93846FDF78DFE4FF400530893C4
S3150800459809950C9508A91F48FDF784FE4FF440783D
S315080045A8CDF82080022609960A950B950C950723BF
S315080045B80D9308A91848FDF775FECDF820800996C9
S315080045C80A960B950C9509230D9308A93846FDF705
S315080045D869FE4FF4C0530893099603230A930B956B
S315080045E80C950A230D9308A90C48FDF75BFED4F829
S315080045F8D83043F00063C4F8D830D4F8D83003F07C
S3150800460800630093009B0EB0BDE8F0810044025891
S315080046180004025800080258000C02580000025804
S3150800462810B5FCF70DFD214C4FF40003A361204893
S31508004638FDF74CFD1F48FDF749FD2046FDF746FDE9
S315080046481D48FDF743FD1D4BD3F8D82022F000621C
S31508004658C3F8D820D3F8EC2022F48072C3F8EC20EB
S31508004668D3F8E82022F48022C3F8E820D3F8E0201B
S3150800467822F00802C3F8E020D3F8E02022F004026A
S31508004688C3F8E020D3F8E02022F00202C3F8E020BD
S31508004698D3F8E02022F00102C3F8E020D3F8F4208A
S315080046A822F00202C3F8F42010BD00BF0004025825
S315080046B8000C025800080258000002580044025824
S315080046C82023038000487047C40400200A23038077
S315080046D800487047E404002008B590F89C32032B7C
S315080046E801D0002008BD01F04DFAFAE708B501F037
S315080046F849FA002008BD08B5084601F077FA0020EF
S3150800470808BD000008B50B7813F0600F06D14B7882
S315080047180A2B14D00B2B17D0062B01D0002008BD66
S315080047284B881B0A212B04D00B491722FBF78FFE4F
S31508004738F4E7CA88172A28BF17220849F6E7012284
S315080047480749FBF784FEE9E78B7813B9044A13602F
S31508004758E4E7FBF7D6FEE1E7CD040020D6040020FF
S315080047681805002010B50446812100F02FF901210B
S31508004778204600F02BF9002010BD000010B50446AD
S3150800478840230222812100F016F940230222012142
S31508004798204600F010F94023034A0121204600F07C
S315080047A83DF9002010BD00BFEC14002000487047F2
S315080047B8EC14002008B500F57171D0F80404FCF76C
S315080047C824FA08BD08B5C1EBC10293000344D3F81F
S315080047D80822D0F80404FCF746FA08BD08B5C1EB68
S315080047E8C102930003449A6CD0F80404FCF785FACE
S315080047F808BD08B5D0F80404FCF72AFB08BD000074
S3150800480810B50446C3684BB1022B01D1012106E055
S315080048189121074800F00AF9012100E00021D4F89F
S315080048280404FCF7FEFAD4F80404FCF7D2FA10BD1F
S31508004838C45D000810B50446D0F80404FCF7F4FA79
S315080048482268D2F8003E43F00103C2F8003E236A04
S3150800485823B1044A136943F006031361FFF762FD9F
S3150800486810BD00BF00ED00E010B50446FFF75BFD7C
S31508004878D4F80404FCF7E1FA10BD08B5D0F8040426
S31508004888FCF7F6FA08BD08B5D0F80404FCF7EEFA02
S3150800489808BD10B504460120FFF743FDD4F8040403
S315080048A8FCF7E8FA10BD10B504460020FFF739FDF5
S315080048B8D4F80404FCF7E0FA10BD000003780BB13D
S315080048C80020704710B503461748C0F80434C3F8E3
S315080048D8C002164B0360092343600222C260002304
S315080048E8036182610122C261036243628362C36211
S315080048F80363FEF79EFE80B90B4C80212046FEF71F
S3150800490815FE402200212046FEF7ECFD80220121F3
S315080049182046FEF7E7FD002010BD4FF493710448C2
S3150800492800F084F8E8E700BF2C15002000000840CE
S31508004938C45D0008D0F8C03211F0800F08D101F024
S315080049487F01C1EBC1018A00134493F8FE01704741
S3150800495801F07F01C1EBC1018A00134493F83E00B8
S31508004968704708B5D0F8C002FFF752FB08BD022801
S3150800497807D8DFE800F00206040000207047012087
S3150800498870470220704708B5D0F8C002FEF72BFF1B
S31508004998FFF7EDFF08BD08B5D0F8C002FEF7E2FE3E
S315080049A8FFF7E5FF08BD08B5D0F8C002FEF7FBFE1D
S315080049B8FFF7DDFF08BD10B51C4613462246D0F89A
S315080049C8C002FFF781FAFFF7D2FF10BD08B5D0F885
S315080049D8C002FFF7B9FAFFF7CAFF08BD08B5D0F84D
S315080049E8C002FFF748FBFFF7C2FF08BD08B5D0F8B5
S315080049F8C002FFF781FBFFF7BAFF08BD08B5D0F874
S31508004A08C002FFF74DFAFFF7B2FF08BD08B5D0F8A0
S31508004A18C002FFF706FBFFF7AAFF08BD08B5D0F8DE
S31508004A28C002FFF7C7FAFFF7A2FF08BD08B500F0EE
S31508004A3805F8FCE708B5FFF76BFC08BD08B5FFF7EE
S31508004A486CFC08BD08B500F0E1FEFFF7F3FF00F0BF
S31508004A58FDFA01F0F7F800F057F800F049F808BD34
S31508004A6808B5FFF7EBFF00F005FB00F061F800F06A
S31508004A7801F808BD08B500F0DFF8012803D00B4B8C
S31508004A881B78012B00D008BD00F002FB084B1B68F9
S31508004A98084A1268134403F5FA739842F3D3034B8A
S31508004AA800221A7000F0B6FEEDE700BF20050020C8
S31508004AB81C05002024050020014B1860704700BF1C
S31508004AC81C050020014B1868704700BF1C0500200C
S31508004AD808B5054B1B78012B00D008BD00F0D8FA9D
S31508004AE8024B1860F9E700BF2005002024050020BE
S31508004AF808B5044B01221A70FFF7EAFFFFF7BAFF59
S31508004B0808BD00BF2005002010B500F005FA00F022
S31508004B18B9FB064C0123237000F0EAFA0023237038
S31508004B2800F064FF0223237010BD00BFEE040020C6
S31508004B3800B583B00DF10701184800F037FC0128C5
S31508004B4810D00DF10701154800F00EFB012812D008
S31508004B580DF10701114800F0C9FF012814D003B068
S31508004B685DF804FB0E4B01221A709DF807100B48D6
S31508004B7800F0F2F9E5E70A4B00221A709DF80710CB
S31508004B88064800F0E9F9E3E7054B02221A709DF892
S31508004B980710024800F0E0F9E1E700BF2805002001
S31508004BA8EE04002008B500F067FF08BD38B50446CE
S31508004BB80D460E4B1B78012B09D00C4B1B7853B1AD
S31508004BC80A4B1B78022B0BD000F0BEF938BDC9B2C8
S31508004BD800F0BAFBF1E7E9B2204600F0A9FAEFE7D8
S31508004BE8E9B2204600F058FFEEE700BFEE040020C1
S31508004BF8074B1B78022B05D0032B05D0012B05D0B4
S31508004C08402070473F2070470020704708207047AB
S31508004C18EE040020074B1B78022B05D0032B05D082
S31508004C28012B05D0402070473F2070470020704769
S31508004C3808207047EE04002008B500F07BF9034603
S31508004C4800B10123184608BD014B00225A70704767
S31508004C5868050020034BFE22DA7018710222A3F8B1
S31508004C68442070476805002010B5054C00232370BA
S31508004C78FFF7EAFFFF23E3700123A4F8443010BDC9
S31508004C8868050020064BFF22DA7000221A71597847
S31508004C9859719A71DA711A720622A3F84420704774
S31508004CA86805002008B50020FFF7D4FF08BD0000F6
S31508004CB8074BFF22DA70074A9A6400221A715A715A
S31508004CC89A710722C3F807200822A3F844207047D8
S31508004CD868050020D05D0008044BFF22DA70426898
S31508004CE89A640122A3F84420704700BF680500208B
S31508004CF808B53120FFF7AEFF08BD000038B5084CE7
S31508004D08FF23E370002525716571FFF771FFA07110
S31508004D18E571257265720723A4F8443038BD00BFCB
S31508004D286805002038B5FFF78FFF0E4C012525705A
S31508004D38FF23E3701023237100236371FFF758FFDD
S31508004D48A071FFF767FFE071FFF764FFC0F307205C
S31508004D5820726572A5720823A4F8443000F072FF21
S31508004D6838BD00BF6805002038B50546FFF740FF7F
S31508004D786A7890420FD90A4CA16C201D00F06AFD8A
S31508004D88FF23E3706A78A36C1344A3646B78013332
S31508004D98A4F8443038BD2220FFF75CFFFAE700BFC5
S31508004DA86805002038B50446FFF722FF637898425D
S31508004DB811D961680A4DA9646278281D00F04AFD70
S31508004DC8FF23EB706278AB6C1344AB6463780133EA
S31508004DD8A5F8443038BD2220FFF73CFFFAE700BFA4
S31508004DE868050020F8B50546174600244E1E39B151
S31508004DF815F8013B1C44E4B2FFF720FE3146F5E7F7
S31508004E083C600120F8BD000010B5084CFF23E3708C
S31508004E18E21D4168A06CFFF7E5FF20710023637166
S31508004E28A3710823A4F8443010BD00BF6805002004
S31508004E3838B505460D4B9C6CFFF7DAFE6A1C411E11
S31508004E48204600F003FF60B1084CFF23E370FFF724
S31508004E58CFFE0138A36C0344A3640123A4F84430A5
S31508004E6838BD3120FFF7F6FEFAE700BF68050020CF
S31508004E7810B50446FFF7BCFE01386378984213DD7F
S31508004E88114BFF22DA700122A3F84420617879B120
S31508004E98A21C0D4B986C00F0D9FE88B161780A4AB5
S31508004EA8936C0B44936410BD2220FFF7D3FEFAE7F0
S31508004EB800F0DCFE0028F6D13120FFF7CBFEF2E73A
S31508004EC83120FFF7C7FEEEE76805002008B54168F8
S31508004ED8074B986C00F0BEFE30B1054BFF22DA701E
S31508004EE80122A3F8442008BD3120FFF7B3FEFAE7EC
S31508004EF86805002008B500F08DFC034BFF22DA7020
S31508004F080122A3F8442008BD6805002008B589B21F
S31508004F18FFF74CFE08BD0000054B00221A709A647C
S31508004F2883F84320A3F844209A705A70704700BF44
S31508004F3868050020034B1B780BB101207047002039
S31508004F48704700BF68050020024B002283F84320FB
S31508004F58704700BF6805002008B50378FF2B23D0E3
S31508004F68354A1278012A2BD1C93B352B53D8DFE8A5
S31508004F7803F04052524F52524C43494652525252EB
S31508004F8852525252525252525252525252525252EB
S31508004F98525252525252525252525252312B282E71
S31508004FA85252523452373A3DFFF7BCFE224B93F819
S31508004FB84330012B33D0204BB3F94410002932DC97
S31508004FC808BDFFF7D1FEF1E7FFF7ECFEEEE7FFF7BE
S31508004FD883FEEBE7FFF718FFE8E7FFF769FEE5E763
S31508004FE8FFF760FEE2E7FFF74DFEDFE7FFF73CFE57
S31508004FF8DCE7FFF71DFFD9E7FFF73AFFD6E7FFF724
S315080050087DFED3E7FFF762FFD0E7FFF773FFCDE72B
S31508005018FFF76EFECAE72020FFF71CFEC6E710203A
S31508005028FFF718FEC7E71846012380F84330033010
S31508005038FFF76CFFC4E700BF68050020024B002293
S315080050481A605A609A60704710E000E008B5FFF7E2
S31508005058F5FF054B054A5A6000229A600521196032
S31508005068034B1A6008BD00BF10E000E0FF520700B6
S31508005078B4050020044B1B6813F4803F03D0034A89
S31508005088136801331360704710E000E0B405002088
S3150800509808B5FFF7EFFF014B186808BDB4050020EF
S315080050A808B5FFF7F5FF08BD054BDB6913F0200FB8
S315080050B804D0034B5B6A03700120704700207047D1
S315080050C80048004010B5094B9862FFF7E1FF00F168
S315080050D80A04064BDB6913F0800F05D1FFF7AEFC0F
S315080050E8FFF7D6FFA042F4D910BD00BF004800401C
S315080050F810B588B00D4C236823F0010323600023FC
S3150800510800934FF4614201920293039304930C228D
S3150800511805920693079369462046FEF7DDF8236845
S3150800512843F00103236008B010BD00BF00480040E3
S3150800513870B506460D4640290ED82846FFF7C2FF21
S315080051480024ABB2A3420CD9FFF778FC305DFFF711
S31508005158B9FF0134A4B2F4E784210248FFF766FCD4
S31508005168EBE770BDD85D000870B5254B1C78BCB94F
S315080051782448FFF799FF012801D0204670BD214B26
S315080051881B78013BDBB23F2BF7D8FFF781FF1E4B95
S3150800519818601E4B00221A70194B01221A70ECE788
S315080051A806460D46194B1B78013316481844FFF76F
S315080051B87BFF0446012815D1144B1A780132D2B25E
S315080051C81A70104B1B789A4201D00024D5E710496B
S315080051D8304600F03FFB0A4B00221A700B4B1B782F
S315080051E82B70CAE7FFF754FF074B1B6864339842CE
S315080051F803D90024024B1C70BFE70024BDE700BF93
S31508005208F9050020B8050020FC050020FA0500204D
S31508005218B9050020F0B4194D2C6D24F040542C65BE
S31508005228002401E00134E4B2112C23D8144D15F8F2
S31508005238146005EB44056F78F51905FB00054FF46E
S31508005248FA5CBCFBF5FC05FB0CF5B5F5FA5FE9D18C
S3150800525835463D4405FB000C4FF4FA55B5FBFCF5FD
S315080052680D80013DADB2B5F5007FDBD216701F7013
S31508005278012000E00020F0BC704700BF0044025837
S31508005288285E000870B58CB00023ADF82E308DF86E
S315080052982D308DF82C300BAB0DF12D020DF12E01AA
S315080052A84FF4FA70FFF7B6FF002842D0234C244B78
S315080052B823600025A560E560012626746574A57433
S315080052C8BDF82E306361A6619DF82D30E3619DF81F
S315080052D82C3023626662A662E66226636563A66365
S315080052E8E563266404236364A564E3642565636546
S315080052F8A565E66525666566A3662046FCF7F4FA9D
S31508005308039504950596069640F2676307930893EE
S31508005318099503A92046FCF731FC00963346022274
S3150800532811462046FCF76DFC2046FCF786FC0CB0B7
S3150800533870BDB8210348FFF779FBB7E700060020D8
S3150800534800A00040005E000810B58AB040F2E1737C
S315080053580193002302930393090404910593069382
S3150800536807930893522309930123024601A90E4875
S31508005378FCF77DFC08B10AB010BD01210A48FCF704
S31508005388ACFC0028F7D1FFF783FE00F132040121AF
S315080053980548FCF781FD0028EDD0FFF74FFBFFF71E
S315080053A877FEA042F3D9E6E70006002030B58BB0B1
S315080053B804460D4640211048FCF777FD10B9002031
S315080053C80BB030BD23466A4640210B48FCF798FCCB
S315080053D868B9009A40F267639A4201D00020EFE75D
S315080053E8019B33B99DF80E302B700120E8E70020A1
S315080053F8E6E70020E4E700BF0006002038B50546C2
S31508005408002401E00134E4B20E2C12D8FFF716FB8B
S3150800541804EB44029300084AD358AB42F2D804EB8B
S3150800542844029100044A0A4452681344AB42E9D933
S3150800543800E0FF24204638BD4C5E000808B5C1F3D5
S31508005448090363B903688B4201D1012008E040F8D3
S31508005458041B4FF4806200F0FDF9012000E00020EB
S3150800546808BD2DE9F04107460068FFF7C7FFFF2882
S3150800547804D14FF000084046BDE8F081FCF780FFEC
S3150800548800264FF0010805E04FF00008B8F1000FB4
S315080054981CD001361F2E19D83D68740125443C4492
S315080054A80434FFF7CBFA224629460120FDF730F8DF
S315080054B850B900231F2BE9D8595DE25CD2B2914254
S315080054C8E2D10133DBB2F5E74FF00008FCF786FFB7
S315080054D8D1E7000070B50E460E4B984212D0054625
S315080054E80D4B994209D10B4C254624B1314628461D
S315080054F8FFF7A4FF58B1204670BDFFF7B2FF20B1E9
S315080055082C46F2E7054C2546EFE70024EDE700248C
S31508005518F1E700BFA40A002000000208A006002040
S315080055282DE9F84306460C4617461D46DFF88480DB
S3150800553801EA08080368B3F1FF3F0AD03368434510
S315080055480ED14FF00109B9F1010F12D04846BDE84E
S31508005558F8834146FFF772FF81460028F3D0EDE746
S3150800556841463046FFF7B6FF0646E8B14FF001094F
S31508005578E9E73368E41A3444043405E017F8013BCC
S3150800558804F8013B013DE1D0FFF758FA331DE31A49
S31508005598B3F5806FF2D308F580613046FFF79AFFB6
S315080055A8064620B1041DE9E74FF00009CEE74FF09B
S315080055B80009CBE700FCFFFF70B586B004460D4628
S315080055C800230093884203D80E2938D8012600E01C
S315080055D8002616B9304606B070BDFCF7D1FE01E0C4
S315080055E80134E4B2AC4227D8FFF728FA1549630014
S315080055F823449A008B188A585B68002B18BFB2F1A7
S31508005608FF3F18D000230193202305930A46630019
S315080056181819810008461144497A02910244137AF6
S31508005628039301230493694601A8FCF7B9FC0028EB
S31508005638D6D0002600E00026FCF7D0FECAE70026EA
S31508005648C8E700BF4C5E00084FF0FF33024A1360F4
S31508005658024A1360704700BFA0060020A40A00206B
S3150800566870B504460D4616464A1E154B1B1A9A422D
S3150800567803D9002001280ED070BDFFF7BFFEFF280A
S3150800568801D10020F8E728190138FFF7B7FEFF28E7
S3150800569814D00120EEE70B4B23400B4A934206D061
S315080056A82B46324621460948FFF73AFFE4E72B46D8
S315080056B8324621460648FFF733FFDDE70020DBE7D9
S315080056C8FFFF1F0800FCFFFF00000208A0060020D5
S315080056D8A40A002070B54A1E0F4B1B1A9A4205D910
S315080056E8FF210E460020012812D070BD05460C463B
S315080056F8FFF784FE064660190138FFF77FFE014664
S31508005708FF2818BFFF2E01D00120ECE70020EAE7A2
S315080057183046FFF751FFE8E7FFFF1F08104B1B68E5
S31508005728B3F1FF3F01D10120704700B583B00C4A99
S31508005738536891680B44D1680B4411690B44516945
S315080057480B4491690B44D26913445B42019301AA3D
S3150800575804210448FFF784FF03B05DF804FB00BF83
S31508005768A40A0020980202080D4B1B680D4A126805
S315080057781A440D4B1B6813440C4A126813440C4A06
S3150800578812681A440B4B1B681A440B4B1B681344C4
S315080057980A4A1268DA4201D1012070470020704788
S315080057A80000020804000208080002080C000208A3
S315080057B810000208140002081800020898020208D5
S315080057C808B50E4B1B68B3F1FF3F07D10C4B1B6896
S315080057D8B3F1FF3F09D10123184608BD0748FFF76B
S315080057E840FE03460028F7D0F0E70548FFF739FEDC
S315080057F803460028F0D00123EEE700BFA40A0020DC
S31508005808A0060020004870470000020808B500F006
S3150800581838FA08BD10B500F021FA00B910BDFEF730
S3150800582869FD0028FAD0FFF7BDF9FBF76FFBFFF70C
S3150800583805FC00F017FA054B0340054A936000F08B
S3150800584811FA446800F01FFAA047E7E780FFFF1F30
S3150800585800ED00E070B50D460446531E9EB23AB1F7
S3150800586815F8013B04F8013BFFF7E8F83246F4E778
S3150800587870BD0000094B03F11801002232B19A7471
S3150800588800225A61064B054A1A6070479A7459618C
S31508005898183318310132D2B2F0E700BFE80E0020FB
S315080058A8180F00200A4B1B6883B110B45C69084AB4
S315080058B8146019749860D86000225A7418600139FF
S315080058C808445860987C5DF8044B7047FF20704779
S315080058D8180F002038B504460D4601281CD8620062
S315080058E82244D100114B0B445A7C1B7C9A4219D08E
S315080058F80E4B0B44DA6815705A7C01325A74DA680A
S315080059080132DA605B689A420ED9084A0846515845
S315080059180244D160012038BD4FF4E1710448FFF70D
S3150800592885F8DCE70020F6E70120F4E7E80E002012
S31508005938005F000808B50146024B1878FFF7CAFF4A
S3150800594808BD00BF1C0F002038B504460D460128BF
S315080059581ED804EB4403DA00124B13445B7CEBB104
S3150800596862002244D1000F4B0B449A6812782A70B9
S315080059785A7C013A5A749A6801329A605B689A4264
S315080059880ED9084A0846515802449160012006E093
S315080059984FF4F2710448FFF749F8DAE7002038BDF2
S315080059A80120FCE7E80E0020005F000808B501465C
S315080059B8024B1878FFF7C8FF08BD00BF600F002024
S315080059C810B50446012806D804EB4404E200054B42
S315080059D81344587C10BD4FF401710348FFF726F8A5
S315080059E8F2E700BFE80E0020005F000838B5FFF7A9
S315080059F841FF1B4C4021601CFFF754FF2070194DCE
S31508005A084021681CFFF74EFF28702378FF2B1DD00E
S31508005A18FF281BD0144C002214492046FBF7ACF883
S31508005A2813492046FBF7D1F80120FEF77AFC2046F1
S31508005A38FBF7D2F8FCF79CFCD4F8C002FEF700FA8C
S31508005A48FFF740F8B0F5FA6F05D338BD8521094840
S31508005A58FEF7ECFFDEE74FF4FA60FFF72DF8F4E7F8
S31508005A681C0F0020600F0020A40F00203C04002013
S31508005A788C040020005F000810B5064CD4F8C00254
S31508005A88FEF7FCF92046FBF78EF80020FEF749FCDE
S31508005A9810BD00BFA40F002070B506460D463F2965
S31508005AA806D82846FFF746FF012806D100240FE046
S31508005AB8BB210D48FEF7BAFFF3E7BF210A48FEF7F0
S31508005AC8B5FFF3E7C8210848FEF7B0FF0134A4B2CA
S31508005AD8ABB2A34207D9FEF7B1FF305DFFF72AFF3D
S31508005AE80128F3D0EEE770BD005F000870B50646DA
S31508005AF80D461F4BD3F8C002FDF72EFF1D4B1C7829
S31508005B089CB91D48FFF752FF012801D0204670BDF1
S31508005B18194B1B78013BDBB23E2BF7D8154B0122F4
S31508005B281A70164B00221A70F0E7144B1B780133CB
S31508005B3811481844FFF73AFF0446012801D0002403
S31508005B48E4E70E4B1A780132D2B21A700A4B1B7860
S31508005B589A4201D00024D9E709493046FFF77AFE68
S31508005B68044B00221A70054B1B782B70CEE700BF32
S31508005B78A40F0020A812002068120020A9120020ED
S31508005B886912002030B583B0144B1878FFF718FF50
S31508005B9808B30546402800D9402500240AE04FF4F2
S31508005BA8A4710F48FEF742FF9DF807200D4B1A55BA
S31508005BB80134E4B2A54208D90DF10701074B187854
S31508005BC8FFF7C2FE0128EFD0E9E7ABB2054A812103
S31508005BD80548FEF71BFF03B030BD00BF1C0F0020A9
S31508005BE8005F0008A80E0020A40F002070B5044620
S31508005BF8FEF7DCFD064621460F48FEF7B2FE85B2DB
S31508005C08002406E04FF4B5710C48FEF70FFF01347F
S31508005C18A4B2AC4207D2315D094B1878FFF75AFE91
S31508005C280128F4D0EEE7FEF7C1FD4023024601211C
S31508005C380148FEF7F3FE70BDA40F0020005F0008B8
S31508005C48600F002008B5FFF7FFFC08BD08B5FFF789
S31508005C5807FD08BD08B5FFF73DFD08BD08B5FFF700
S31508005C6883FD08BD08B5FFF7CDFD08BD08B5FFF7E4
S31508005C7855FD034608B9184608BDFFF7A1FD0346B2
S31508005C88F9E772B6704762B670470A44914200F15E
S31508005C98FF3300D1704710B511F8014B03F8014FCF
S31508005CA89142F9D110BD0000F8B500BFF8BC08BC90
S31508005CB89E467047F8B500BFF8BC08BC9E467047B4
S31508005CC800000000000000000000000000000000BE
S31508005CD800000000010000000200000003000000A8
S31508005CE80400000000000000050000000000000095
S31508005CF80000000000000000060000000000000088
S31508005D080000000000000000070000000000002056
S31508005D18000000000102030401020304060708093B
S31508005D28000000000102030401020304060708092B
S31508005D380001020304050607080C10141820304051
S31508005D480100000002000000040000000600000030
S31508005D58080000000A0000000C00000010000000FF
S31508005D68200000004000000080000000000100003C
S31508005D7844656661756C740057696E5553422042CE
S31508005D88756C6B20496E7465726661636500000000
S31508005D984F70656E424C54205573657200000000BA
S31508005DA857696E5553422042756C6B20446576696F
S31508005DB8636500006D61696E2E6300007573626421
S31508005DC85F636F6E662E63004F70656E424C5400B3
S31508005DD82E2E2F2E2E2F2E2E2F536F757263652F6C
S31508005DE841524D434D375F53544D333248372F721E
S31508005DF8733233322E6300002E2E2F2E2E2F2E2E80
S31508005E082F536F757263652F41524D434D375F5354
S31508005E18544D333248372F63616E2E6300000000F5
S31508005E2805020602060307030803090309040A0408
S31508005E380B040C040C050D050E050F050F061006B8
S31508005E4810071008000002080000020001010000FF
S31508005E58000004080000020002010000000006080D
S31508005E680000020003010000000008080000020004
S31508005E780401000000000A080000020005010000ED
S31508005E8800000C08000002000601000000000E08C9
S31508005E9800000200070100000000100800000200C8
S31508005EA800020000000012080000020001020000BB
S31508005EB8000014080000020002020000000016088C
S31508005EC80000020003020000000018080000020093
S31508005ED80402000000001A0800000200050200007B
S31508005EE800001C08000002000602000000001E0848
S31508005EF800000200070200002E2E2F2E2E2F2E2E0F
S31508005F082F536F757263652F41524D434D375F5353
S31508005F18544D333248372F7573622E6300000000DC
S30D08005F2821030008BD02000870
S30908005F3099020008BC
S31508005F3400000000EC02002054030020BC030020EB
S31508005F44000000000000000000000000000000003F
S31508005F54000000000000000000000000000000002F
S31508005F64000000000000000000000000000000001F
S31508005F74000000000000000000000000000000000F
S31508005F8400000000000000000000000000000000FF
S31508005F9400000000000000000000000000000000EF
S31508005FA400000000000000000000000000000000DF
S31508005FB400000000000000000000000000000000CF
S31508005FC400000000000000000000000000000000BF
S31508005FD400000000000000000100000000000000AE
S31508005FE40E33CDAB34126DE6ECDE05000B00000073
S31508005FF4000000000000000000000000000000008F
S31508006004000000000000000000000000000000007E
S31508006014000000000000000000000000000000006E
S31508006024000000000000000000000000000000005E
S315080063540000000000000000AC1200200090D003EA
S315080063640090D003010000001000000071410008ED
S315080063747D4100082D42000809420008F54100083D
S31508006384494200086D42000812010002000000405C
S31508006394501DAC6000020102030100000403090455
S315080063A41A030000000000000000000000000000BE
S315080063B400000000000000000000000085470008F7
S315080063C46D4700080D4700080000000000000000A3
S315080063D4F5460008FF460008E146000800000000EC
S315080063E40000000000000000C94600080000000084
S315080063F4D546000809022000010100C0320904003C
S315080064040002FF000000070581024000FF0705019E
S31508006414024000FF0A0600020000004001000400D2
S70508000405E9
